:100000000C945E010C94F51F0C94CA1F0C949F1F56
:100010000C94741F0C94491F0C941E1F0C94F31E17
:100020000C94C81E0C9491010C9491010C949101B4
:100030000C9491010C9491010C9491010C949101F8
:100040000C9491010C9491010C9491010C949101E8
:100050000C9491010C9491010C9491010C947E1ECE
:100060000C9491010C94481E0C941E1E0C9491014A
:100070000C9491010C9491010C9491010C9420200A
:100080000C9491010C9491010C9491010C949101A8
:100090000C9491010C9491010C9491010C94910198
:1000A0000C9491010C9491010C9491010C94910188
:1000B0000C9491010C9491010C9491010C94910178
:1000C0000C9491010C9491010C9491010C94910168
:1000D0000C9491010C9491010C9491010C94910158
:1000E0000C9491010C9448030C94E2030C94360395
:1000F0000C944E030C94AD1A0C94D91B0C945B0415
:100100000C94ED1A0C9429020C94C9030C9433043A
:100110000C94221C0C94141B0C9452030C94130387
:100120000C9444030C94DB200C94F1010C945104C6
:100130000C9432030C941A040C94F4030C94C00134
:100140000C94CF010C94C1030C94E3010C94B704FC
:100150000C947B020C9417030C94FC020C943D0449
:100160000C94E71B0C94EE1A0C94531B0C94400354
:100170000C94D8030C941B030C94FC030C940604FD
:100180000C9410040C943A030C9428030C94381C1F
:100190000C9422030C9401030C9493010C94CE0351
:1001A0000C942C030C94EC030C941F030C94470444
:1001B0000C94290400002100240027002A002D00AF
:1001C0003000330001010000040107010A010000B2
:1001D0002200250028002B002E00310034000201EF
:1001E0000000050108010B010505050507050808C4
:1001F0000808020202020A0A0808040404040101B1
:1002000001010101010103030303030303030407C5
:1002100007070C0C0C0C0C0C0C0C0202020206065C
:100220000606060606060B0B0B0B0B0B0B0B01024F
:1002300010202008081020401020408002010201F8
:1002400008040201010204081020408080402010B0
:100250000804020180040201804020100804020109
:100260000804020101020408102040800102040871
:100270001020408000000A0B02090C0D0E08070335
:100280000401000000000000000000000000000069
:10029000000000000000000000000000000000005E
:1002A000121110000000000000000000000000001B
:1002B00000000000000000000000DB202092F11C84
:1002C00011241FBECFEFD1E2DEBFCDBF00E00CBFD7
:1002D00012E0A0E0B2E0E6E3FDE500E00BBF02C003
:1002E00007900D92A83AB107D9F72CE1A8EAB2E03D
:1002F00001C01D92A13FB207E1F711E0CEE5D1E0C8
:1003000000E006C021970109802FFE010E949C2C6D
:10031000CD35D10780E00807A9F70E9430210C9461
:10032000992E0C940000AF92BF92CF92DF92EF9281
:10033000FF920F931F93CF93DF936C017B018B018F
:10034000040F151FEB015E01AE18BF08C017D107DF
:1003500059F06991D601ED91FC910190F081E02D69
:10036000C6011995892B79F7C501DF91CF911F91AE
:100370000F91FF90EF90DF90CF90BF90AF900895D6
:10038000FC01538D448D252F30E0842F90E0821B9B
:10039000930B541710F0CF96089501970895FC0120
:1003A000918D828D981761F0A28DAE0FBF2FB11D78
:1003B0005D968C91928D9F5F9F73928F90E00895D0
:1003C0008FEF9FEF0895FC01918D828D981731F08A
:1003D000828DE80FF11D858D90E008958FEF9FEFDE
:1003E0000895FC01918D228D892F90E0805C9F4FB4
:1003F000821B91098F739927089581E39CE10E94E4
:10040000F10121E0892B09F420E0822F0895FC01FD
:10041000A48DA80FB92FB11DA35ABF4F2C91848D65
:1004200090E001968F739927848FA689B7892C93C2
:10043000A089B1898C91837080648C93938D848D15
:10044000981306C00288F389E02D80818F7D808318
:100450000895EF92FF920F931F93CF93DF93EC01D8
:1004600081E0888F9B8D8C8D98131AC0E889F9895B
:10047000808185FF15C09FB7F894EE89FF8960835E
:10048000E889F98980818370806480839FBF81E0DF
:1004900090E0DF91CF911F910F91FF90EF90089521
:1004A000F62E0B8D10E00F5F1F4F0F731127E02EFC
:1004B0008C8D8E110CC00FB607FCFACFE889F98934
:1004C000808185FFF5CFCE010E940702F1CFEB8D31
:1004D000EC0FFD2FF11DE35AFF4FF0829FB7F89408
:1004E0000B8FEA89FB8980818062CFCF682F81E3FF
:1004F0009CE10C942902CF93DF93EC01888D882333
:10050000B9F0AA89BB89E889F9898C9185FD03C076
:10051000808186FD0DC00FB607FCF7CF8C9185FF5B
:10052000F2CF808185FFEDCFCE010E940702E9CF97
:10053000DF91CF91089580E090E0892B29F00E940F
:10054000FD0181110E94000080E090E0892B49F0BC
:1005500080E090E0892B29F00E94000081110E9428
:10056000000080E090E0892B49F080E090E0892B4A
:1005700029F00E94000081110E94000080E090E0BC
:10058000892B49F080E090E0892B29F00E9400003F
:1005900081110C9400000895282F30E0F901EC58E7
:1005A000FD4F9491F901E25DFD4F449128513E4F7A
:1005B000F9012491222309F435C0992311F19150B6
:1005C0009231F8F4E92FF0E08827E651FD4F8F4F84
:1005D0000C949C2C1B031F03FC0213031703010341
:1005E000220328032C03320336033A034003440357
:1005F000010348034E035203809180008F7780935C
:100600008000E22FF0E0EE0FFF1FE253FE4FA591B6
:10061000B4918FB7F894EC91611148C040954E2386
:100620004C938FBF0895809180008F7DE8CF80919B
:100630008000877FE4CF84B58F7784BDE2CF84B517
:100640008F7DFBCF8091B0008F778093B000D9CFA2
:100650008091B0008F7DF9CF809190008F7780934B
:100660009000CFCF809190008F7DF9CF8091900046
:10067000877FF5CF8091A0008F778093A000C1CFB6
:100680008091A0008F7DF9CF8091A000877FF5CF6A
:10069000809120018F7780932001B3CF809120013A
:1006A0008F7DF9CF80912001877FF5CF4E2BB8CF7A
:1006B000CF93DF9390E0FC01E25DFD4F24918851E0
:1006C0009E4FFC0184918823D1F090E0880F991F00
:1006D000FC01EC54FE4FA591B491FC01E253FE4F96
:1006E000C591D49161110EC09FB7F8948C91E22FFF
:1006F000E0958E238C932881E223E8839FBFDF91CE
:10070000CF9108958FB7F894EC91E22BEC938FBFC3
:10071000F6CF1F93CF93DF93182FEB0161E00E9478
:100720005803209739F460E0812FDF91CF911F911A
:100730000C94CC02CF3FD10511F461E0F5CFE12F4D
:10074000F0E0EC58FD4FE491E150E23108F0B3C025
:10075000F0E08827E155FC4F8F4F0C949C2CC1038F
:10076000C903CE03D803E2035B04EC03F403FC03E8
:10077000060410041A04290433045B043D044704EE
:10078000510484B5806884BDC7BDDF91CF911F91AE
:10079000089584B5806284BDC8BDF7CF8091800084
:1007A000806880938000D0938900C0938800EDCF4B
:1007B00080918000806280938000D0938B00C093F2
:1007C0008A00E3CF80918000886080938000D0937E
:1007D0008D00C0938C00D9CF8091B0008068809349
:1007E000B000C093B300D1CF8091B00080628093FD
:1007F000B000C093B400C9CF80919000806880930E
:100800009000D0939900C0939800BFCF8091900042
:10081000806280939000D0939B00C0939A00B5CFE4
:1008200080919000886080939000D0939D00C09349
:100830009C00ABCF8091A00080688093A000809145
:10084000A0008F7B8093A000D093A900C093A80044
:100850009CCF8091A00080628093A000D093AB00D9
:10086000C093AA0092CF8091A00088608093A000DE
:10087000D093AD00C093AC0088CF809120018068F8
:1008800080932001D0932901C09328017ECF8091CD
:100890002001806280932001D0932B01C0932A0114
:1008A00074CF80912001886080932001D0932D0126
:1008B000C0932C016ACFC038D1050CF03ECF33CFA6
:1008C0003FB7F8948091B6029091B702A091B80218
:1008D000B091B90226B5A89B05C02F3F19F001962B
:1008E000A11DB11D3FBFBA2FA92F982F8827BC018A
:1008F000CD01620F711D811D911D42E0660F771FB2
:10090000881F991F4A95D1F708958F929F92AF92B1
:10091000BF92CF92DF92EF92FF924B015C010E9457
:1009200060046B017C010E9460046C197D098E09D2
:100930009F09683E734081059105A8F321E0821A62
:100940009108A108B10888EEC80E83E0D81EE11C0A
:10095000F11C81149104A104B10429F7FF90EF90D8
:10096000DF90CF90BF90AF909F908F9008950895A3
:100970008091000C9091010CA091020CB091030C9D
:10098000892B8A2B8B2BE1F08091FC0B9091FD0B36
:10099000A091FE0BB091FF0B892B8A2B8B2B81F042
:1009A00080911602909117028F3F910549F0809136
:1009B000FA0B9091FB0B892B19F0109213020895FA
:1009C00081E0809313020895CF93DF9380EC90E051
:1009D0000E94760290E080E00E947602C0E0D4E0BF
:1009E0002091AA023091AB02CE0180509440821730
:1009F0009307A8F46991603C51F48BED90E00E945C
:100A000076026CED81E39CE10E942902E9CF6B3D07
:100A1000C9F78BED90E00E9476026DEDF3CF80EC8C
:100A200090E00E9476021092AB021092AA02DF912F
:100A3000CF91089580EC90E00E94760283E090E0F0
:100A40000E9476026091160281E39CE10E942902D5
:100A500080EC90E00C94760280EC90E00E947602AC
:100A600085E090E00E9476026091140281E39CE1AF
:100A70000E94290280EC90E00C94760280EC90E0D9
:100A80000E94760284E090E00E9476026091FA0B68
:100A900081E39CE10E94290280EC90E00C947602B4
:100AA000CF93C82F80EC90E00E94760280E990E01E
:100AB0000E9476026C2F81E39CE10E94290280EC67
:100AC00090E0CF910C947602803C51F48BED90E055
:100AD0000E9476028CED682F81E39CE10C94290240
:100AE0008B3DC9F78BED90E00E9476028DEDF3CF40
:100AF0001F93CF93DF9380EC90E00E94760281E019
:100B000090E00E947602C091000CD091010C1091EF
:100B1000020C8091030C0E946405812F0E946405E1
:100B20008D2F0E9464058C2F0E94640580EC90E05C
:100B3000DF91CF911F910C9476021F93CF93DF9397
:100B400080EC90E00E94760282E090E00E947602C3
:100B5000C091FC0BD091FD0B1091FE0B8091FF0B0F
:100B60000E946405812F0E9464058D2F0E946405F8
:100B70008C2F0E94640580EC90E0DF91CF911F9153
:100B80000C94760280EC90E00E94760284E290E081
:100B90000E9476028091A9020E94640580EC90E098
:100BA0000C947602CF93C0910102C35680EC90E082
:100BB0000E94760283E290E00E9476028C2F0E94CF
:100BC000640580EC90E0CF910C94760260E08DE0BB
:100BD0000C94CC0261E08DE00C94CC02CF93DF93B7
:100BE000EC0161E08DE00E94CC020E94E60564E623
:100BF00070E080E090E00E9485040E94EA0564E6CF
:100C000070E080E090E00E948504219771F7DF9109
:100C1000CF910C94E60560E08CE00C94CC020F932D
:100C20001F93CF93DF938C01EC01892B11F4C1E06A
:100C3000D0E00E940B0664E670E080E090E00E9445
:100C4000850461E08CE00E94CC0264E670E080E004
:100C500090E00E9485040115110559F3219749F789
:100C6000DF91CF911F910F910C940B060E94EA0522
:100C70000E940B066AE070E080E090E00E9485042C
:100C800061E08CE00E94CC020E94E60565E070E025
:100C900080E090E00E948504E9CF0F931F93CF93EB
:100CA000DF938C01EC01892B11F4C1E0D0E061E00D
:100CB0008CE00E94CC0260E08DE00E94CC0264E6F1
:100CC00070E080E090E00E94850460E08CE00E948B
:100CD000CC0261E08DE00E94CC0264E670E080E02E
:100CE00090E00E9485040115110509F32197F9F69A
:100CF0000E940B06DF91CF911F910F910C94E60596
:100D00002F923F924F925F926F927F928F929F921B
:100D1000AF92BF92CF92DF92EF92FF920F931F9309
:100D2000CF93DF93CDB7DEB7C857D1090FB6F8948C
:100D3000DEBF0FBECDBFE9969FAF8EAFE9971A0118
:100D4000DC0118960D911D912D913C911B97619698
:100D50000CAF1DAF2EAF3FAF61971C960D911D914B
:100D60002D913C911F9709831A832B833C835096C6
:100D70000D911D912D913C9153970D831E832F83CF
:100D8000388754960D911D912D913C915797098765
:100D90001A872B873C87E6966FAFE697E7967FAF7B
:100DA000E797A85ABF4F6396BFAFAEAF6397FC01FA
:100DB000E45AFF4F6596FFAFEEAF65978C01005A7E
:100DC0001F4F67961FAF0EAF67979C012C593F4F7F
:100DD00069963FAF2EAF699788599F4F6B969FAF2B
:100DE0008EAF6B97E996AEADBFADE997A459BF4FF3
:100DF0006D96BFAFAEAF6D97E996EEADFFADE997DB
:100E0000E059FF4F6F96FFAFEEAF6F97E9960EADCB
:100E10001FADE9970C581F4FA1961FAF0EAFA197BA
:100E2000E9962EAD3FADE99728583F4FA3963FAFC7
:100E30002EAFA397E9968EAD9FADE99784589F4F4B
:100E4000A5969FAF8EAFA597E996AEADBFADE997DA
:100E5000A058BF4FA796BFAFAEAFA797E996EEAD2C
:100E6000FFADE997EC57FF4FA996FFAFEEAFA997FB
:100E7000E9960EAD1FADE99708571F4FAB961FAF10
:100E80000EAFAB97E9962EAD3FADE99724573F4F94
:100E9000AD963FAF2EAFAD97E9968EAD9FADE9977A
:100EA00080579F4FAF969FAF8EAFAF97E996AEAD8D
:100EB000BFADE997AC56BF4FE196BFAFAEAFE1977C
:100EC000E796AEADBFADE7970D911D912D913C9189
:100ED0000D871E872F87388B6396EEADFFAD639726
:100EE000008311832283338361968CAD9DADAEADBB
:100EF000BFAD619788589B45A549B842800F911FA7
:100F0000A21FB31F4D815E816F81788509851A8587
:100F10002B853C85402751276227732709811A8139
:100F20002B813C81402351236223732309851A8539
:100F30002B853C854027512762277327840F951FF7
:100F4000A61FB71F8C019D0147E0000F111F221F34
:100F5000331F4A95D1F7AC01BD01E9E1769567955C
:100F600057954795EA95D1F7402B512B622B732B60
:100F700089819A81AB81BC81480F591F6A1F7B1FF1
:100F8000E796AEADBFADE79714960D911D912D91EB
:100F90003C911797098B1A8B2B8B3C8B6596EEAD8A
:100FA000FFAD6597008311832283338389859A85FA
:100FB000AB85BC858A5A9844A843B741800F911FDE
:100FC000A21FB31FC980DA80EB80FC800D811E81D7
:100FD0002F813885C026D126E226F326C422D522C9
:100FE000E622F722C026D126E226F3268C0D9D1D8F
:100FF000AE1DBF1D8C019D01FCE0000F111F221FC3
:10100000331FFA95D1F76C017D01A4E1F694E794C2
:10101000D794C794AA95D1F7C02AD12AE22AF32AF5
:10102000C40ED51EE61EF71EE796AEADBFADE79720
:1010300018968D919D910D90BC91A02D8D8B9E8BBE
:10104000AF8BB88F6796EEADFFAD679780839183C6
:10105000A283B3838D819E81AF81B88585529F48DD
:10106000AF4DBB4D0D891E892F89388D800F911F83
:10107000A21FB31F49805A806B807C80442655266E
:10108000662677264C205D206E207F2009811A81FC
:101090002B813C814026512662267326840D951DA6
:1010A000A61DB71D8C019D01EFE03695279517957C
:1010B0000795EA95D1F72C013D01F1E1440C551C4F
:1010C000661C771CFA95D1F7402A512A622A732AA6
:1010D0004C0C5D1C6E1C7F1CE796AEADBFADE79758
:1010E0001C968D919D910D90BC91A02D898F9A8F0A
:1010F000AB8FBC8F6996EEADFFAD6997808391830E
:10110000A283B38389819A81AB81BC81825191434F
:10111000A244BE43098D1A8D2B8D3C8D800F911FEB
:10112000A21FB31F8A019B010C251D252E253F25DB
:1011300004211521262137210427152726273727A3
:10114000800F911FA21FB31F4C015D011AE0B694DE
:10115000A794979487941A95D1F78C019D0186E105
:10116000000F111F221F331F8A95D1F70829192953
:101170002A293B29040D151D261D371DE796AEAD06
:10118000BFADE79750968D919D910D90BC91A02D8C
:101190008D8F9E8FAF8FB8A36B96EEADFFAD6B9723
:1011A00080839183A283B3838155904FA348BA4033
:1011B000840F951FA61FB71FB701A601442555250B
:1011C0006625772540235123622373234C255D2513
:1011D0006E257F25840F951FA61FB71F4C015D014B
:1011E00047E0880C991CAA1CBB1C4A95D1F7AC019E
:1011F000BD01E9E17695679557954795EA95D1F751
:10120000482959296A297B29400F511F621F731FE2
:10121000E796AEADBFADE79754968D919D910D9039
:10122000BC91A02D89A39AA3ABA3BCA36D96EEADF0
:10123000FFAD6D9780839183A283B383865D9943CD
:10124000A847B84B8C0D9D1DAE1DBF1D73016201DB
:10125000C026D126E226F326C422D522E622F72292
:10126000C424D524E624F7248C0D9D1DAE1DBF1D7E
:101270004C015D01FCE0880C991CAA1CBB1CFA9572
:10128000D1F76C017D01A4E1F694E794D794C7945B
:10129000AA95D1F7C828D928EA28FB28C40ED51E5C
:1012A000E61EF71EE796AEADBFADE79758968D9157
:1012B0009D910D90BC91A02D8DA39EA3AFA3B8A727
:1012C0006F96EEADFFAD6F9780839183A283B3835A
:1012D0008D5E994BAF4CB745840D951DA61DB71D6E
:1012E0002801390144265526662677264C205D20A4
:1012F0006E207F204026512662267326840D951D80
:10130000A61DB71D4C015D01EFE0B694A79497941C
:101310008794EA95D1F72C013D01F1E1440C551C6D
:10132000661C771CFA95D1F7482859286A287B282B
:101330004C0C5D1C6E1C7F1CE796AEADBFADE797F5
:101340005C968D919D910D90BC91A02D89A79AA737
:10135000ABA7BCA7A196EEADFFADA197808391830B
:10136000A283B3838F5F9A46A94BB240800F911F2F
:10137000A21FB31F8A019B010C251D252E253F2589
:101380000421152126213721042715272627372751
:10139000800F911FA21FB31F4C015D011AE0B6948C
:1013A000A794979487941A95D1F78C019D0186E1B3
:1013B000000F111F221F331F8A95D1F70829192901
:1013C0002A293B29040D151D261D371DE796AEADB4
:1013D000BFADE79790968D919D910D90BC91A02DFA
:1013E0008DA79EA7AFA7B8ABA396EEADFFADA39711
:1013F00080839183A283B38388529746AF47B649CF
:10140000840F951FA61FB71FB701A60144255525B8
:101410006625772540235123622373234C255D25C0
:101420006E257F25840F951FA61FB71F4C015D01F8
:1014300047E0880C991CAA1CBB1C4A95D1F7AC014B
:10144000BD01E9E17695679557954795EA95D1F7FE
:10145000482959296A297B29400F511F621F731F90
:10146000E796AEADBFADE79794968D919D910D90A7
:10147000BC91A02D89AB9AABABABBCABA596EEAD46
:10148000FFADA59780839183A283B3838155984054
:10149000AB4BB4478C0D9D1DAE1DBF1D730162018A
:1014A000C026D126E226F326C422D522E622F72240
:1014B000C424D524E624F7248C0D9D1DAE1DBF1D2C
:1014C0004C015D01FCE0880C991CAA1CBB1CFA9520
:1014D000D1F76C017D01A4E1F694E794D794C79409
:1014E000AA95D1F7C828D928EA28FB28C40ED51E0A
:1014F000E61EF71EE796AEADBFADE79798968D91C5
:101500009D910D90BC91A02D8DAB9EABAFABB8AFB4
:10151000A796EEADFFADA79780839183A283B38397
:101520008F54944AA109B109840D951DA61DB71DBC
:101530002801390144265526662677264C205D2051
:101540006E207F204026512662267326840D951D2D
:10155000A61DB71D4C015D01EFE0B694A7949794CA
:101560008794EA95D1F72C013D01F1E1440C551C1B
:10157000661C771CFA95D1F7482859286A287B28D9
:101580004C0C5D1C6E1C7F1CE796AEADBFADE797A3
:101590009C968D919D910D90BC91A02D89AF9AAF95
:1015A000ABAFBCAFA996EEADFFADA9978083918399
:1015B000A283B38382549842A34AB647800F911FF7
:1015C000A21FB31F8A019B010C251D252E253F2537
:1015D00004211521262137210427152726273727FF
:1015E000800F911FA21FB31F4C015D011AE0B6943A
:1015F000A794979487941A95D1F78C019D0186E161
:10160000000F111F221F331F8A95D1F708291929AE
:101610002A293B29040D151D261D371DE796AEAD61
:10162000BFADE797D0968D919D910D90BC91A02D67
:1016300021968CAF9DAFAEAFBFAF2197AB96EEAD0D
:10164000FFADAB9780839183A283B3834C015D018F
:10165000FEED8F1AFEEE9F0AFFE6AF0AF4E9BF0A1D
:10166000840E951EA61EB71EB701A601442555255A
:101670006625772540235123622373234C255D255E
:101680006E257F25480D591D6A1D7B1D4A015B0192
:1016900097E0880C991CAA1CBB1C9A95D1F7E9E12C
:1016A0007695679557954795EA95D1F74829592931
:1016B0006A297B29400F511F621F731FE796AEAD49
:1016C000BFADE797D4968D919D910D90BC91A02DC3
:1016D00025968CAF9DAFAEAFBFAF2597AD96EEAD63
:1016E000FFADAD9780839183A283B3834C015D01ED
:1016F000FDE68F1AFEE89F0AF7E6AF0AF2E0BF0A9E
:101700008C0C9D1CAE1CBF1C73016201C026D1262F
:10171000E226F326C422D522E622F722C424D524C9
:10172000E624F724C80CD91CEA1CFB1C460157010F
:10173000FCE0880C991CAA1CBB1CFA95D1F7A4E10B
:10174000F694E794D794C794AA95D1F7C828D928D6
:10175000EA28FB28C40ED51EE61EF71EE796AEAD9E
:10176000BFADE797D8968D919D910D90BC91A02D1E
:1017700029968CAF9DAFAEAFBFAF2997AF96EEADB8
:10178000FFADAF9780839183A283B3834C015D014A
:10179000F2E78F1AFCEB9F0AF6E8AF0AF9E5BF0AF9
:1017A000840C951CA61CB71C28013901442655261B
:1017B000662677264C205D206E207F20402651260D
:1017C00062267326480C591C6A1C7B1C530142017B
:1017D000BFE0B694A79497948794BA95D1F781E126
:1017E000440C551C661C771C8A95D1F7482859284B
:1017F0006A287B284C0C5D1C6E1C7F1CE796AEADE6
:10180000BFADE797DC968D919D910D90BC91A02D79
:101810002D968CAF9DAFAEAFBFAF2D97E196EEADDD
:10182000FFADE19780839183A283B3834C015D0177
:10183000FFED8F1AF7EF9F0AFBE4AF0AF6EBBF0A42
:10184000800E911EA21EB31E8A019B010C251D2530
:101850002E253F2504211521262137210427152770
:1018600026273727080D191D2A1D3B1D4801590140
:101870009AE0B694A794979487949A95D1F7E6E165
:10188000000F111F221F331FEA95D1F708291929CC
:101890002A293B29040D151D261D371D89889A8884
:1018A000AB88BC888EE9881A8AED980A81EEA80A6E
:1018B00089E0B80A840E951EA61EB71EB301A201C8
:1018C00040275127622773274C215D216E217F21FC
:1018D0004425552566257725480D591D6A1D7B1D14
:1018E0004A015B01F5E0880C991CAA1CBB1CFA9507
:1018F000D1F7ABE17695679557954795AA95D1F7BE
:10190000482959296A297B29400F511F621F731FDB
:101910008DA09EA0AFA0B8A490EC891A9CE4990A6F
:101920009FEBA90A9FE3B90A8C0C9D1CAE1CBF1C3F
:1019300068017901C426D526E626F726C420D520DD
:10194000E620F720C026D126E226F326C80CD91CB3
:10195000EA1CFB1C46015701B9E0880C991CAA1C23
:10196000BB1CBA95D1F787E1F694E794D794C79456
:101970008A95D1F7C828D928EA28FB28C40ED51E95
:10198000E61EF71E89AC9AACABACBCACAFEA8A1AC7
:10199000A5EA9A0AA1EAAA0AA9EDBA0A840C951C3A
:1019A000A61CB71C2A013B014C245D246E247F2415
:1019B000402251226222732244265526662677262B
:1019C000480C591C6A1C7B1C530142019EE0880C88
:1019D000991CAA1CBB1C9A95D1F7E2E176946794F6
:1019E00057944794EA95D1F7482859286A287B28C4
:1019F0004C0C5D1C6E1C7F1C8D849E84AF84B8884B
:101A0000B6E58B1AB8E39B0AB9E4AB0AB6E1BB0AA8
:101A1000800E911EA21EB31E970186010425152576
:101A20002625372504231523262337230C251D259A
:101A30002E253F25080D191D2A1D3B1D4801590162
:101A4000FCE0B694A79497948794FA95D1F7A4E113
:101A5000000F111F221F331FAA95D1F7082919293A
:101A60002A293B29040D151D261D371D89A09AA082
:101A7000ABA0BCA0E3EA8E1AEFEE9E0AE0EDAE0A40
:101A8000E9E2BE0A840E951EA61EB71EB301A2018E
:101A900040275127622773274C215D216E217F212A
:101AA0004425552566257725480D591D6A1D7B1D42
:101AB0004A015B01B5E0880C991CAA1CBB1CBA95B5
:101AC000D1F78BE176956795579547958A95D1F72C
:101AD000482959296A297B29400F511F621F731F0A
:101AE0008DA89EA8AFA8B8ACFDEA8F1AFBEE9F0A9E
:101AF000FBEBAF0AFDEFBF0A8C0C9D1CAE1CBF1C9C
:101B000068017901C426D526E626F726C420D5200B
:101B1000E620F720C026D126E226F326C80CD91CE1
:101B2000EA1CFB1C4601570199E0880C991CAA1C71
:101B3000BB1C9A95D1F7E7E1F694E794D794C79444
:101B4000EA95D1F7C828D928EA28FB28C40ED51E63
:101B5000E61EF71E2D968CAC9DACAEACBFAC2D979F
:101B60008FE7881A89E1980A8EE5A80A87E2B80A01
:101B7000840C951CA61CB71C2A013B014C245D2437
:101B80006E247F244022512262227322442655264D
:101B900066267726480C591C6A1C7B1C530142019F
:101BA000FEE0880C991CAA1CBB1CFA95D1F7A2E197
:101BB0007694679457944794AA95D1F74828592862
:101BC0006A287B284C0C5D1C6E1C7F1C8D8C9E8CA7
:101BD000AF8CB8A098E3891A94E0990A9CE2A90A0C
:101BE00098E1B90A800E911EA21EB31E97018601CC
:101BF00004251525262537250423152326233723D9
:101C00000C251D252E253F25080D191D2A1D3B1DC0
:101C100048015901BCE0B694A79497948794BA956B
:101C2000D1F784E1000F111F221F331F8A95D1F7CE
:101C3000082919292A293B29040D151D261D371DA0
:101C400089A89AA8ABA8BCA8AAE18A1AA2E39A0A12
:101C5000AEE1AA0AAEEDBA0A840E951EA61EB71E04
:101C6000B301A20140275127622773274C215D2130
:101C70006E217F214425552566257725480D591D60
:101C80006A1D7B1D4A015B0195E0880C991CAA1C0A
:101C9000BB1C9A95D1F7EBE17695679557954795DB
:101CA000EA95D1F7482959296A297B29400F511F04
:101CB000621F731F29968CAC9DACAEACBFAC29974C
:101CC000BAE28B1AB8EF9B0AB8ECAB0ABCE3BB0ACA
:101CD0008C0C9D1CAE1CBF1C68017901C426D52646
:101CE000E626F726C420D520E620F720C026D126F8
:101CF000E226F326C80CD91CEA1CFB1C460157013E
:101D0000F9E0880C991CAA1CBB1CFA95D1F7A7E135
:101D1000F694E794D794C794AA95D1F7C828D92800
:101D2000EA28FB28C40ED51EE61EF71E898C9A8C65
:101D3000AB8CBC8CE9E78E1AE2EF9E0AEAE2AE0AAF
:101D4000EBE0BE0A840C951CA61CB71C2A013B01C3
:101D50004C245D246E247F2440225122622273226F
:101D60004426552666267726480C591C6A1C7B1C7F
:101D700053014201BEE0880C991CAA1CBB1CBA95F9
:101D8000D1F782E176946794579447948A95D1F776
:101D9000482859286A287B284C0C5D1C6E1C7F1C27
:101DA0008DA49EA4AFA4B8A8F3E18F1AFBEE9F0AFE
:101DB000F5EAAF0AFAEBBF0A800E911EA21EB31E0F
:101DC000970186010425152526253725042315238B
:101DD000262337230C251D252E253F25080D191DEB
:101DE0002A1D3B1D480159019CE0B694A794979485
:101DF00087949A95D1F7E4E1000F111F221F331F3A
:101E0000EA95D1F7082919292A293B29040D151D1E
:101E1000261D371D25968CAC9DACAEACBFAC25976E
:101E20008BEF881A86E1980A8CE1A80A86E5B80A41
:101E3000840E951EA61EB71EB301A201402751278E
:101E4000622773274C215D216E217F214425552572
:101E500066257725480D591D6A1D7B1D4A015B01CA
:101E6000F5E0880C991CAA1CBB1CFA95D1F7ABE1D4
:101E70007695679557954795AA95D1F74829592999
:101E80006A297B29400F511F621F731F8D889E880E
:101E9000AF88B88C98E0891A9CE5990A90E1A90A64
:101EA00093E0B90A8C0C9D1CAE1CBF1C6801790123
:101EB000C426D526E626F726C420D520E620F7201E
:101EC000C026D126E226F326C80CD91CEA1CFB1C2E
:101ED00046015701B9E0880C991CAA1CBB1CBA9595
:101EE000D1F787E1F694E794D794C7948A95D1F710
:101EF000C828D928EA28FB28C40ED51EE61EF71EDE
:101F000089A49AA4ABA4BCA4A7E28A1AADEF9A0A4A
:101F1000A0E9AA0AA8E9BA0A840C951CA61CB71C59
:101F20002A013B014C245D246E247F24402251224F
:101F3000622273224426552666267726480C591CB1
:101F40006A1C7B1C530142019EE0880C991CAA1C50
:101F5000BB1C9A95D1F7E2E1769467945794479425
:101F6000EA95D1F7482859286A287B284C0C5D1C33
:101F70006E1C7F1C4601570184249524A624B72497
:101F800021968CAD9DADAEADBFAD21978657934BDD
:101F9000A54DB247800F911FA21FB31F9501840169
:101FA00004231523262337230C251D252E253F2505
:101FB000800F911FA21FB31F8C019D01FCE036957D
:101FC000279517950795FA95D1F7E5960CAF1DAFB4
:101FD0002EAF3FAFE5978C019D01A4E1000F111FCB
:101FE000221F331FAA95D1F7E5968CAD9DADAEADFE
:101FF000BFADE597082B192B2A2B3B2B040D151D84
:10200000261D371D89A19AA1ABA1BCA18E5B964C60
:10201000A540B109840F951FA61FB71F80269126E2
:10202000A226B326880E991EAA1EBB1ED501C40186
:1020300044E0880F991FAA1FBB1F4A95D1F75CE1A6
:10204000B694A794979487945A95D1F7882A992A99
:10205000AA2ABB2A800E911EA21EB31E4DA55EA504
:102060006FA578A94F5759406E4878474C0D5D1DB4
:102070006E1D7F1D73016201C026D126E226F32664
:10208000C824D924EA24FB24C40ED51EE61EF71E5C
:10209000B701A601EBE0440F551F661F771FEA95B5
:1020A000D1F7F5E1F694E794D794C794FA95D1F770
:1020B000C42AD52AE62AF72AC80CD91CEA1CFB1C1C
:1020C00049AD5AAD6BAD7CAD4E5D5E49624672491D
:1020D000440E551E661E771EB901A80148255925D4
:1020E0006A257B254C255D256E257F25440E551ED2
:1020F000661E771ED20123013D014C0C5D1C6E1C37
:102100007F1C29964CAD5DAD6EAD7FAD2997445FC8
:10211000574C6A417240400F511F621F731F950157
:1021200084010C251D252E253F2504251525262552
:102130003725040F151F261F371FB901A801A9E075
:102140007695679557954795AA95D1F7B7E1000F12
:10215000111F221F331FBA95D1F7042B152B262BE5
:10216000372B040D151D261D371D49895A896B898A
:102170007C894C5B554161447B45480D591D6A1D66
:102180007B1D4601570184249524A624B72480266C
:102190009126A226B326840E951EA61EB71EB50153
:1021A000A40184E0440F551F661F771F8A95D1F75D
:1021B0009CE1B694A794979487949A95D1F7842A32
:1021C000952AA62AB72A800E911EA21EB31E4D8DF7
:1021D0005E8D6F8D78A1475550436142744BC40E9C
:1021E000D51EE61EF71EB301A20140275127622724
:1021F0007327482559256A257B254C0D5D1D6E1DCD
:102200007F1DDB01CA01EBE0880F991FAA1FBB1FCE
:10221000EA95D1F7F5E17695679557954795FA9543
:10222000D1F7482B592B6A2B7B2B480D591D6A1D62
:102230007B1DC9A4DAA4EBA4FCA4B0EACB1AB4EBCE
:10224000DB0AB4E4EB0AB9E0FB0A4C0C5D1C6E1C23
:102250007F1C68017901C824D924EA24FB24C42600
:10226000D526E626F7264C0C5D1C6E1C7F1CF20161
:1022700023013F01440E551E661E771ECDA8DEA821
:10228000EFA8F8ACF0E9CF1AF3E4DF0AF0E4EF0AC4
:10229000F1E4FF0AC00ED11EE21EF31E9501840177
:1022A0000427152726273727042515252625372512
:1022B0000C0D1D1D2E1D3F1D68017901A9E0F6942E
:1022C000E794D794C794AA95D1F7B7E1000F111FEF
:1022D000221F331FBA95D1F70C291D292E293F291A
:1022E000040D151D261D371D2596CCACDDACEEACBE
:1022F000FFAC25978AE3C81A81E8D80A84E6E80A81
:1023000087EDF80AC80CD91CEA1CFB1C4A015B01CA
:1023100084249524A624B72480269126A226B326B9
:102320008C0C9D1CAE1CBF1C7501640184E0CC0CA0
:10233000DD1CEE1CFF1C8A95D1F79CE1B694A79496
:10234000979487949A95D1F78C289D28AE28BF281A
:10235000800E911EA21EB31ECD84DE84EF84F88809
:1023600096E0C91A98EDD90A9EE5E90A95E1F90ABD
:10237000C40ED51EE61EF71EB301A2014027512749
:1023800062277327482559256A257B254C0D5D1D3D
:102390006E1D7F1D6A017B01EBE0CC0CDD1CEE1C89
:1023A000FF1CEA95D1F7F5E1769567955795479526
:1023B000FA95D1F74C295D296E297F29480D591DC1
:1023C0006A1D7B1DC98CDA8CEB8CFC8CABE7CA1ABE
:1023D000AFECDA0AA0E1EA0AABE2FA0A4C0C5D1CA7
:1023E0006E1C7F1C68017901C824D924EA24FB24CF
:1023F000C426D526E626F7264C0C5D1C6E1C7F1CD9
:10240000F20123013F01440E551E661E771ECDA02A
:10241000DEA0EFA0F8A4FBEFCF1AF2EEDF0AF7E799
:10242000EF0AFBEFFF0AC00ED11EE21EF31E95015C
:102430008401042715272627372704251525262557
:1024400037250C0D1D1D2E1D3F1D68017901A9E0CA
:10245000F694E794D794C794AA95D1F7B7E1000F03
:10246000111F221F331FBA95D1F70C291D292E29C0
:102470003F29040D151D261D371DC9A8DAA8EBA894
:10248000FCA887ECC81A8FE2D80A8BE2E80A86E239
:10249000F80AC80CD91CEA1CFB1C4A015B01842405
:1024A0009524A624B72480269126A226B3268C0C38
:1024B0009D1CAE1CBF1C7501640184E0CC0CDD1CAE
:1024C000EE1CFF1C8A95D1F79CE1B694A7949794D3
:1024D00087949A95D1F78C289D28AE28BF28800E26
:1024E000911EA21EB31E2196CCACDDACEEACFFACAF
:1024F00021979BE1C91A96E6D90A94E2E90A99E183
:10250000F90AC40ED51EE61EF71EB301A20140272C
:10251000512762277327482559256A257B254C0DAD
:102520005D1D6E1D7F1D6A017B01EBE0CC0CDD1C87
:10253000EE1CFF1CEA95D1F7F5E176956795579566
:102540004795FA95D1F74C295D296E297F29480DC9
:10255000591D6A1D7B1D2D96CCACDDACEEACFFACDD
:102560002D97A8E0CA1AA3E8DA0AADE5EA0AA0EEB8
:10257000FA0A4C0C5D1C6E1C7F1C68017901C82492
:10258000D924EA24FB24C426D526E626F7264C0CBB
:102590005D1C6E1C7F1CF20123013F01440E551E81
:1025A000661E771ECD88DE88EF88F88CFBE9CF1A8F
:1025B000F9EADF0AF3E5EF0AFBE3FF0AC00ED11EDA
:1025C000E21EF31E950184010427152726273727CD
:1025D00004251525262537250C0D1D1D2E1D3F1DF7
:1025E00068017901A9E0F694E794D794C794AA9575
:1025F000D1F7B7E1000F111F221F331FBA95D1F792
:102600000C291D292E293F29040D151D261D371DB6
:10261000CD84DE84EF84F8888CEBC81A8DEDD80A5F
:1026200086EDE80A8BE0F80AC80CD91CEA1CFB1CF2
:102630004A015B0180949094A094B094802A912ADE
:10264000A22AB32A84249524A624B7248C0C9D1C8A
:10265000AE1CBF1C7501640186E0CC0CDD1CEE1CB9
:10266000FF1C8A95D1F79AE1B694A7949794879422
:102670009A95D1F78C289D28AE28BF28800E911EF0
:10268000A21EB31EC9A4DAA4EBA4FCA499E6C91A3D
:10269000D10895EDE90A9CEBF90AC40ED51EE61E99
:1026A000F71EB301A2014095509560957095482999
:1026B00059296A297B2940275127622773274C0D06
:1026C0005D1D6E1D7F1D6A017B01EAE0CC0CDD1CE7
:1026D000EE1CFF1CEA95D1F7F6E1769567955795C4
:1026E0004795FA95D1F74C295D296E297F29480D28
:1026F000591D6A1D7B1D2996CCACDDACEEACFFAC40
:102700002997A9E5CA1AACEDDA0AABE6EA0AA4E50C
:10271000FA0AC40CD51CE61CF71C280139014094A8
:10272000509460947094442A552A662A772A482443
:1027300059246A247B244C0C5D1C6E1C7F1C730185
:102740006201AFE0CC0CDD1CEE1CFF1CAA95D1F79A
:10275000B1E17694679457944794BA95D1F74C2891
:102760005D286E287F28440E551E661E771EC9A060
:10277000DAA0EBA0FCA0B7ECCB1ABFE5DB0ABCE605
:10278000EB0AB3E0FB0AC00ED11EE21EF31E950158
:102790008401009510952095309504291529262946
:1027A000372904271527262737270C0D1D1D2E1D19
:1027B0003F1D680179018BE0F694E794D794C794A4
:1027C0008A95D1F795E1000F111F221F331F9A95AB
:1027D000D1F70C291D292E293F29040D151D261D71
:1027E000371D2196CCACDDACEEACFFAC2197EDE310
:1027F000CE1AE6EADE0AE4EAEE0AEAE9FE0AC80CC4
:10280000D91CEA1CFB1C4A015B0180949094A094A3
:10281000B094802A912AA22AB32A84249524A6243B
:10282000B7248C0C9D1CAE1CBF1C75016401E6E036
:10283000CC0CDD1CEE1CFF1CEA95D1F7FAE1B69436
:10284000A79497948794FA95D1F78C289D28AE2861
:10285000BF28800E911EA21EB31EC98CDA8CEB8C91
:10286000FC8CFEE6CF1AF3E3DF0AF3EFEF0AF0E7A2
:10287000FF0AC40ED51EE61EF71EB301A201409545
:10288000509560957095482959296A297B294027D8
:102890005127622773274C0D5D1D6E1D7F1D6A0138
:1028A0007B01AAE0CC0CDD1CEE1CFF1CAA95D1F725
:1028B000B6E17695679557954795BA95D1F74C2926
:1028C0005D296E297F29480D591D6A1D7B1DCDA8E4
:1028D000DEA8EFA8F8AC83E8C81A8BE0D80A80E13C
:1028E000E80AF108C40CD51CE61CF71C28013901C4
:1028F0004094509460947094442A552A662A772A0A
:10290000482459246A247B244C0C5D1C6E1C7F1CBB
:10291000730162018FE0CC0CDD1CEE1CFF1C8A955C
:10292000D1F791E176946794579447949A95D1F7AB
:102930004C285D286E287F28440E551E661E771E83
:10294000C988DA88EB88FC889FE2C91A92EAD90A1A
:102950009BE7E90A9AE7F90AC00ED11EE21EF31EB0
:10296000950184010095109520953095042915292D
:102970002629372904271527262737270C0D1D1D43
:102980002E1D3F1D68017901EBE0F694E794D79482
:10299000C794EA95D1F7F5E1000F111F221F331FED
:1029A000FA95D1F70C291D292E293F29040D151D53
:1029B000261D371DCDA4DEA4EFA4F8A8A1EBCA1AEA
:1029C000A1E8DA0AA7E5EA0AA0E9FA0AC80CD91CC4
:1029D000EA1CFB1C4A015B0180949094A094B09483
:1029E000802A912AA22AB32A84249524A624B724D3
:1029F0008C0C9D1CAE1CBF1C75016401A6E0CC0CA8
:102A0000DD1CEE1CFF1CAA95D1F7BAE1B694A79481
:102A100097948794BA95D1F78C289D28AE28BF2823
:102A2000800E911EA21EB31E2D968CAD9DADAEAD37
:102A3000BFAD2D9780529941A34DB140840F951F92
:102A4000A61FB71FB301A2014095509560957095E0
:102A5000482959296A297B2940275127622773274A
:102A6000840F951FA61FB71F6C017D014AE0CC0C97
:102A7000DD1CEE1CFF1C4A95D1F7AC01BD01E6E15F
:102A80007695679557954795EA95D1F74C295D2935
:102A90006E297F29480D591D6A1D7B1D8DA19EA1A0
:102AA000AFA1B8A58C5E9C4BAE4FBC45840D951D67
:102AB000A61DB71D2801390140945094609470946C
:102AC000442A552A662A772A482459246A247B24D2
:102AD000840D951DA61DB71D6C017D01FFE0CC0C7A
:102AE000DD1CEE1CFF1CFA95D1F72C013D01A1E184
:102AF0007694679457944794AA95D1F74C285D280B
:102B00006E287F28440E551E661E771E25968CADB6
:102B10009DADAEADBFAD25978F559E4EA74FB14B26
:102B2000800F911FA21FB31F95018401009510957E
:102B3000209530950429152926293729042715279A
:102B400026273727800F911FA21FB31F6C017D011D
:102B50001BE0F694E794D794C7941A95D1F78C01AB
:102B60009D0185E1000F111F221F331F8A95D1F7A8
:102B70000C291D292E293F29040D151D261D371D41
:102B80008D8D9E8DAF8DB8A18E579148AC4AB840BF
:102B9000880D991DAA1DBB1D4A015B01809490946C
:102BA000A094B094802A912AA22AB32A842495243E
:102BB000A624B724880D991DAA1DBB1D6C017D019B
:102BC000E6E0CC0CDD1CEE1CFF1CEA95D1F74C01B5
:102BD0005D01FAE1B694A79497948794FA95D1F79A
:102BE0008C289D28AE28BF28800E911EA21EB31EE1
:102BF00089AD9AADABADBCAD8B5C9D40A54CB244EC
:102C0000840F951FA61FB71FB301A20140955095D1
:102C100060957095482959296A297B2940275127B1
:102C200062277327840F951FA61FB71F6C017D01B4
:102C30004AE0CC0CDD1CEE1CFF1C4A95D1F7AC0120
:102C4000BD01E6E17695679557954795EA95D1F7E9
:102C50004C295D296E297F29480D591D6A1D7B1D50
:102C60008D899E89AF89B88D85549D42A842B54D06
:102C7000840D951DA61DB71D28013901409450945F
:102C800060947094442A552A662A772A4824592445
:102C90006A247B24840D951DA61DB71D6C017D0142
:102CA000FFE0CC0CDD1CEE1CFF1CFA95D1F72C01CB
:102CB0003D01A1E17694679457944794AA95D1F782
:102CC0004C285D286E287F28440E551E661E771EF0
:102CD00089A99AA9ABA9BCA98F569C42A947B4411E
:102CE000800F911FA21FB31F9501840100951095BD
:102CF00020953095042915292629372904271527D9
:102D000026273727800F911FA21FB31F6C017D015B
:102D10001BE0F694E794D794C7941A95D1F78C01E9
:102D20009D0185E1000F111F221F331F8A95D1F7E6
:102D30000C291D292E293F29040D151D261D371D7F
:102D400061968CAD9DADAEADBFAD6197880D991DFF
:102D5000AA1DBB1D61968CAF9DAFAEAFBFAF619793
:102D600089819A81AB81BC81800F911FA21FB31F03
:102D700089839A83AB83BC830D811E812F81388523
:102D8000040D151D261D371D0D831E832F833887C7
:102D900089859A85AB85BC85840F951FA61FB71FB3
:102DA00089879A87AB87BC87E796AEADBFADE797BB
:102DB000A05CBF4FE796BFAFAEAFE797B0E42B1A6A
:102DC000310811F00C94600761960CAD1DAD2EAD6D
:102DD0003FAD6197E996AEADBFADE99718960D93FB
:102DE0001D932D933C931B9709811A812B813C8164
:102DF0001C960D931D932D933C931F970D811E815F
:102E00002F81388550960D931D932D933C935397A6
:102E100009851A852B853C8554960D931D932D931A
:102E20003C935797E7968EAD9FADE797C858DF4F15
:102E30000FB6F894DEBF0FBECDBFDF91CF911F91CB
:102E40000F91FF90EF90DF90CF90BF90AF909F9049
:102E50008F907F906F905F904F903F902F9008954C
:102E60000F931F93CF93DF93EC01062F142F60E095
:102E70008E850E94CC023C852D858091AD028823F1
:102E800081F09FB7F8948091AD02813081F58DB3C8
:102E90008093A8024DB38091AC02809584238DBBB2
:102EA0009FBF3CBD2DBD0EBD00000DB407FEFDCF84
:102EB0008EB51EBD00000DB407FEFDCF1EB580917E
:102EC000AD02882351F09FB7F8942091AD02809114
:102ED000A802213079F48DBB9FBF61E08E850E94EE
:102EE000CC02812FDF91CF911F910F910895909384
:102EF000A802D7CF8FBFF1CFAF92BF92CF92DF9210
:102F0000EF92FF920F931F93CF936093E31C709304
:102F1000E41C8093E51C9093E61C6B017C01FF0C84
:102F2000CC08DC2C76019B01AC016C2D7C2D8C2D0A
:102F30009C2D03E10E94352DA12CE8E4BE2EF8EE75
:102F4000CF2EDD24D394E12CF12C00E010E00E9480
:102F5000D82CC22FC22ED32E7A01A701662777273D
:102F600066E88FEC9CE10E94301777276F2D5E2D6D
:102F70004D2D67E88FEC9CE10E9430174C2F68E8DC
:102F80008FEC9CE1CF911F910F91FF90EF90DF901C
:102F9000CF90BF90AF900C94301740E861E88FEC71
:102FA0009CE10E9430179FB7F8948091AE0288236D
:102FB00019F081508093AE028091AE02811105C05C
:102FC0008CB58F7B8CBD1092AD029FBF1092301CD0
:102FD000089540E00C943017CF92DF92EF92FF9269
:102FE0000F931F93CF93DF936AE18FEC9CE10E94D4
:102FF000E917C82FD0E069E18FEC9CE10E94E91746
:10300000682F880F770B880B990B0E94D02A20E03D
:1030100030E040E85EE30E942F2B0E94662C6B019B
:103020008B016091E31C7091E41C8091E51C9091F0
:10303000E61C0E94D02A24ED30E843E45EE40E94BE
:10304000C92ABE0187FD10C06D59710917FF0FC055
:103050006C0D7D1DCB01DF91CF911F910F91FF90E2
:10306000EF90DF90CF900895645A7109EFCF072E4B
:10307000000C880B990B0E94D02A20EB32E748E81D
:103080005FE30E942F2B0E94662CE4CF43E861E8A7
:103090008FEC9CE10E94301762E18FEC9CE10E9472
:1030A000E91783FFF9CF48E062E98FEC9CE10E94C9
:1030B000301781E090E00895CF92DF92EF92FF9277
:1030C0006EE18FEC9CE10E94E91782958F70CC2411
:1030D000C394D12C02C0CC0CDD1C8A95E2F70D2CD8
:1030E000000CEE08FF086DE18FEC9CE10E94E917EF
:1030F00090E044E0959587954A95E1F78A309105EF
:1031000034F5FC01EE0FFF1FE80FF91FEC5DFD4FDA
:10311000608171818281082E000C990B28EE33E0CA
:1031200040E050E00E94032CC701B6010E94032C2E
:10313000213131054105510574F04CE066EA8FEC10
:103140009CE1FF90EF90DF90CF900C94301760E0FF
:1031500070E0CB01E3CF44E0F1CFCF93DF93EC01FC
:10316000863091052CF08D30910534F5069731F5B8
:1031700045EC61EB8FEC9CE10E9430174CE067EB73
:103180008FEC9CE10E943017C6E0D0E06EE18FEC3E
:103190009CE10E94E9178F7094E0CC0FDD1F9A9597
:1031A000E1F74C2F482B6EE98FEC9CE10E94301721
:1031B000DF91CF910C945C18CCE0D0E043EC61EB54
:1031C0008FEC9CE10E9430174AE067EB8FEC9CE1AA
:1031D0000E943017DBCFCF93DF93EC01099714F0F7
:1031E000C8E0D0E06DE18FEC9CE10E94E917C530AA
:1031F000D10514F4C5E0D0E02497CC0FDD1F482F93
:10320000417F4C2B6DE98FEC9CE1DF91CF910C94C9
:1032100030171092EA1C1092E91C6DE18FEC9CE1D2
:103220000E94E917482F4E7F6DE98FEC9CE10C94CA
:10323000301781E090E09093EA1C8093E91C6DE1E7
:103240008FEC9CE10E94E917482F41606DE98FECFB
:103250009CE10C943017CF93DF93EC0141E861E8D7
:103260008FEC9CE10E943017CD2B99F00E94191928
:1032700040E06DE88FEC9CE10E94301740E062EA8C
:103280008FEC9CE10E94301781E090E0DF91CF91BC
:1032900008950E940919ECCF0F931F93CF93DF93EA
:1032A00066E08FEC9CE10E94E917D82F67E08FEC75
:1032B0009CE10E94E917C82F68E08FEC9CE10E9416
:1032C000E9174C2F50E070E060E0762F652F542F07
:1032D00044276D2B8A019B01082BC901B80120E00E
:1032E00038E448EE51E00E94AB2C03E10E94502DDF
:1032F0002093000C3093010C4093020C5093030C6C
:10330000DF91CF911F910F910895CF92DF92EF92AD
:10331000FF92CF93DF936091FC0B7091FD0B809136
:10332000FE0B9091FF0B0E94D02A6B017C0120E0E4
:1033300030EC43EF55E40E94C92AD0E0C0E01816F3
:103340000CF065C020E030E842E256E4C701B60167
:103350000E94C92AC1E0D0E018160CF058C020E045
:1033600030EC43E756E4C701B6010E94C92AC2E027
:10337000D0E018160CF04BC020E030E842EA56E4EA
:10338000C701B6010E94C92AC3E0D0E018160CF0AC
:103390003EC020E034E244EF56E4C701B6010E948B
:1033A000C92AC4E0D0E0181694F520E034EE42E2D9
:1033B00057E4C701B6010E94C92AC5E0D0E018163B
:1033C00034F520E034E244E757E4C701B6010E9437
:1033D000C92AC6E0D0E01816D4F420E034E244EF65
:1033E00057E4C701B6010E94C92AC7E0D0E0181609
:1033F00074F420E034E244E758E4C701B6010E94C7
:10340000C92AC9E0D0E0181614F0C8E0D0E06DE198
:103410008FEC9CE10E94E9178F7044E0CC0FDD1F18
:103420004A95E1F74C2F482B6DE98FEC9CE10E9407
:1034300030170E945C188091301C882319F16DE1CF
:103440008FEC9CE10E94E91790E034E09595879518
:103450003A95E1F78A309105E4F4FC01EE0FFF1F85
:10346000E80FF91FEC5DFD4F80819181A2810A2E4A
:10347000000CBB0B8093FC0B9093FD0BA093FE0BF9
:10348000B093FF0BDF91CF91FF90EF90DF90CF9043
:10349000089580E090E0DC01EDCF68E18FEC9CE1E5
:1034A0000E94E9179FB7F8944091F5095091F609E9
:1034B0006091F7097091F8099FBF4093F909509303
:1034C000FA096093FB097093FC0980FF2AC081E030
:1034D0008093B3028093B2028093B1028091AF02D5
:1034E0009091B0022091B302211108C02091B20244
:1034F000211104C02091B102222301F18F309105E6
:10350000B8F401969093B0028093AF0281E080936B
:103510002D1C80912C1C8823F1F061E08CE00C9430
:10352000CC021092B3021092B2021092B102D6CF26
:1035300081E080932D1C80932C1CEBCF009741F0F1
:1035400001979093B0028093AF0210922D1CE1CFAF
:1035500010922C1CFACF0C940B06CF93DF9362E1F0
:103560008FEC9CE10E94E917C82F482F62E98FEC8D
:103570009CE10E943017C5FD2DC01092E81C1092EE
:10358000E71C8091E91C9091EA1C62E2892B09F406
:1035900063E18FEC9CE10E94E917C82FD0E060E165
:1035A0008FEC9CE10E94E917482F6DE88FEC9CE1BD
:1035B0000E943017E091EB1CF091EC1C309711F059
:1035C000CE01199540E06DE88FEC9CE1DF91CF9141
:1035D0000C943017DF91CF91089508950F931F93A6
:1035E000CF93DF93EC01E881F9810084F185E02D30
:1035F0001995892BB1F06DE0CE010E94E917082FD3
:1036000060E0CE010E94E917182F402F6DE8CE012F
:103610000E943017812F90E0DF91CF911F910F9181
:1036200008958FEF9FEFF8CFCF93DF93EC01E88100
:10363000F9810084F185E02D1995892B69F0888D39
:10364000998D0196998F888F60E0CE010E94E917CD
:1036500090E0DF91CF9108958FEF9FEFFACFCF9356
:10366000DF93EC012097E1F021978091AA029091DD
:10367000AB02843F9140A0F48FEC9CE10E94141BAC
:103680002091AA023091AB02A9014F5F5F4F509386
:10369000AB024093AA0220503C4FF9018083E2CF55
:1036A000DF91CF9108950F931F93CF93DF93EC0198
:1036B0008091F90B811178C08FEC9CE10E94141B62
:1036C00021974091000280FF55C09C0154E0359540
:1036D00027955A95E1F72F7033274F3FD1F4109279
:1036E000AB021092AA02209300020E94EC17909362
:1036F00002028093010269E18FEC9CE10E94E917CC
:103700008093A902CE01DF91CF911F910F910C946C
:103710002F1B2413E4CF0E94EC172091010230915B
:103720000202820F931F97FD0196959587959093BE
:103730000202809301020091A90210E069E18FEC7E
:103740009CE10E94E917800F912F911D9595879517
:103750008093A902CE010E942F1B8FEF809300025D
:103760000E94D2050E94C205DF91CF911F910F9157
:103770000C94E4044F3F39F01092AB021092AA026D
:103780008FEF809300020E94EC17909302028093C7
:10379000010269E18FEC9CE10E94E9178093A90284
:1037A000CE010E942F1BDCCF1092AB021092AA0216
:1037B000EACFCF93DF93EC0163E10E94E91790E039
:1037C000288D398D821B930BDF91CF910895AF9295
:1037D000BF92CF92DF92FF920F931F93CF93DF930D
:1037E0006C015B01EA0162E20E94E917F82E90E0A9
:1037F0009C012C0F3D1F2F3F310529F020F0CFEF0A
:10380000D0E0C81BD90B8501AC0EBD1E0A151B05E7
:1038100041F0F80141918F0160E8C6010E94301724
:10382000F5CF4C2F4F0D62EAC6010E943017CE0132
:10383000DF91CF911F910F91FF90DF90CF90BF90BC
:10384000AF900895CF93DF931F92CDB7DEB7698312
:10385000DC01ED91FC910280F381E02D41E050E02C
:10386000BE016F5F7F4F19950F90DF91CF91089543
:1038700090E080E008950C94ED2BCF938091F70BAE
:10388000811103C00E9409190CC0C091F80BCC2310
:10389000C9F30E9419194C2F62EA8FEC9CE10E9437
:1038A000301745E861E88FEC9CE1CF910C9430171C
:1038B0008091301C882341F18091BA02843A89F4C6
:1038C00040911602509117024F30510514F04EE00E
:1038D00050E057FD40E0406769E88FEC9CE10C94B4
:1038E0003017893A89F440911602509117024231FB
:1038F000510514F041E150E04230510514F442E02A
:1039000050E042504068E8CF0895CF92DF92EF92A6
:10391000FF92CF93DF930E94B804D091301CD11155
:103920007DC080911302811184C1C0912B1CCC23D6
:1039300009F47FC1C090000CD090010CE090020C03
:10394000F090030C61E08091DD1C0E94580361E05F
:103950008091DD1C0E94CC028091DF1C9091E01CC4
:103960008F3F9807C9F061E00E94580360E08091A2
:10397000DF1C0E94CC026AE070E080E090E00E94D0
:10398000850461E08091DF1C0E94CC026AE070E057
:1039900080E090E00E948504DFB7F8948091AE0249
:1039A000811127C0EDE1F2E08491E3E6F2E0949129
:1039B000E82FF0E0EE0FFF1FEC54FE4FA591B491FD
:1039C000EC91E92321F461E085E30E94CC0261E0FF
:1039D00085E30E9458038CB580618CBD8CB58064F2
:1039E0008CBD61E084E30E94580361E083E30E94A0
:1039F00058038091AE028F5F8093AE02DFBF62E416
:103A00008FEC9CE10E94E917823181F081E00E94F5
:103A1000500590E080E00E944D06D0E08D2FDF91B0
:103A2000CF91FF90EF90DF90CF90089540E861E84C
:103A30008FEC9CE10E943017C701B6010E947C17F1
:103A400040E06EE88FEC9CE10E94301740E06FE8A8
:103A50008FEC9CE10E9430176CE08FEC9CE10E949F
:103A6000E917482F43606CE88FEC9CE10E94301707
:103A700044E066EA8FEC9CE10E94301740E869E878
:103A80008FEC9CE10E94301741E861E88FEC9CE1EB
:103A90000E94301781E08093301C0E94581C0E94C5
:103AA00085198091FA0B9091FB0B0E94AD188091C3
:103AB0001402909115020E94EB180E944C196EE1BD
:103AC0008FEC9CE10E94E917482F44606EE98FEC6F
:103AD0009CE10E94301783E59BE19093EC1C80935E
:103AE000EB1C60E08091E11C0E94580340E060EC18
:103AF0008FEC9CE10E9430172091E11C3091E21C78
:103B000080E02230310551F081E02330310531F081
:103B1000C9014297049788F487E1821B2FB7F89474
:103B20008230E9F160F4882309F43FC0813071F0FC
:103B300082E08093AD0280E00AC08FEFEFCF843047
:103B400091F178F18530A1F788E001C080E2909191
:103B5000AC02892B8093AC028091AD02811103C02D
:103B600081E08093AD022FBF2091E11C3091E21CD7
:103B700022303105E1F48DEA9AE1909304028093BA
:103B8000030280916A00836080936A00EC9A0E942D
:103B90003D1C83E090E00E940F06DC2F3FCF81E0C8
:103BA000D6CF82E0D4CF84E0D2CF80E1D0CF233013
:103BB000310569F48DEA9AE190930602809305023B
:103BC00080916A008C6080936A00ED9AE0CFC90111
:103BD00042970497E0F687E1821BE82FF0E0EE0FB2
:103BE000FF1FED5FFD4F2DEA3AE1318320838430E2
:103BF00091F08530B9F0833039F0809169008360AD
:103C000080936900E89AC3CF809169008C608093AB
:103C10006900E99ABCCF8091690080638093690054
:103C2000EA9AB5CF80916900806C80936900EB9A25
:103C3000AECF83E090E00E94EE05F0CE1F920F928F
:103C40000FB60F9211240BB60F922F933F934F9301
:103C50005F936F937F938F939F93AF93BF93EF93F4
:103C6000FF9381E39CE10E940702FF91EF91BF91D6
:103C7000AF919F918F917F916F915F914F913F9104
:103C80002F910F900BBE0F900FBE0F901F901895A5
:103C90001F920F920FB60F9211240BB60F922F9313
:103CA0008F939F93EF93FF93E091411CF091421CFF
:103CB0008081E091471CF091481C82FD1DC09081DD
:103CC00080914A1C8F5F8F7320914B1C821741F0AB
:103CD000E0914A1CF0E0EF5CF34E958F80934A1C14
:103CE000FF91EF919F918F912F910F900BBE0F90AD
:103CF0000FBE0F901F9018958081F2CF1F920F92E8
:103D00000FB60F9211242F933F938F939F93AF93EE
:103D1000BF938091F5099091F609A091F709B091B0
:103D2000F8093091B50223E0230F2D3758F501969D
:103D3000A11DB11D2093B5028093F5099093F6095A
:103D4000A093F709B093F8098091B6029091B70259
:103D5000A091B802B091B9020196A11DB11D809346
:103D6000B6029093B702A093B802B093B902BF9184
:103D7000AF919F918F913F912F910F900FBE0F9018
:103D80001F90189526E8230F0296A11DB11DD2CFD2
:103D90001F920F920FB60F9211240BB60F922F9312
:103DA0003F934F935F936F937F938F939F93AF93C3
:103DB000BF93EF93FF93E0911102F09112021995D6
:103DC000FF91EF91BF91AF919F918F917F916F91F3
:103DD0005F914F913F912F910F900BBE0F900FBEAF
:103DE0000F901F9018951F920F920FB60F921124EB
:103DF0000BB60F922F933F934F935F936F937F93E5
:103E00008F939F93AF93BF93EF93FF93E0910F0234
:103E1000F09110021995FF91EF91BF91AF919F9191
:103E20008F917F916F915F914F913F912F910F9063
:103E30000BBE0F900FBE0F901F9018951F920F9200
:103E40000FB60F9211240BB60F922F933F934F93FF
:103E50005F936F937F938F939F93AF93BF93EF93F2
:103E6000FF93E0910502F09106021995FF91EF9101
:103E7000BF91AF919F918F917F916F915F914F9182
:103E80003F912F910F900BBE0F900FBE0F901F9080
:103E900018951F920F920FB60F9211240BB60F9226
:103EA0002F933F934F935F936F937F938F939F9342
:103EB000AF93BF93EF93FF93E0910302F09104025D
:103EC0001995FF91EF91BF91AF919F918F917F9144
:103ED0006F915F914F913F912F910F900BBE0F907B
:103EE0000FBE0F901F9018951F920F920FB60F9252
:103EF00011240BB60F922F933F934F935F936F93C1
:103F00007F938F939F93AF93BF93EF93FF93E09132
:103F10000D02F0910E021995FF91EF91BF91AF91B3
:103F20009F918F917F916F915F914F913F912F91D1
:103F30000F900BBE0F900FBE0F901F9018951F9201
:103F40000F920FB60F9211240BB60F922F933F933F
:103F50004F935F936F937F938F939F93AF93BF9391
:103F6000EF93FF93E0910B02F0910C021995FF91F2
:103F7000EF91BF91AF919F918F917F916F915F91E1
:103F80004F913F912F910F900BBE0F900FBE0F904E
:103F90001F9018951F920F920FB60F9211240BB617
:103FA0000F922F933F934F935F936F937F938F93D2
:103FB0009F93AF93BF93EF93FF93E0910902F0912A
:103FC0000A021995FF91EF91BF91AF919F918F9147
:103FD0007F916F915F914F913F912F910F900BBE09
:103FE0000F900FBE0F901F9018951F920F920FB653
:103FF0000F9211240BB60F922F933F934F935F9321
:104000006F937F938F939F93AF93BF93EF93FF93A0
:10401000E0910702F09108021995FF91EF91BF918D
:10402000AF919F918F917F916F915F914F913F9150
:104030002F910F900BBE0F900FBE0F901F901895F1
:104040001F920F920FB60F9211240BB60F922F935F
:104050003F934F935F936F937F938F939F93AF9310
:10406000BF93CF93EF93FF938091B402811127C048
:1040700081E08093B402C4E181E39CE10E94F101FC
:10408000892BD9F08FB7F8944091271C5091281CA8
:104090002091231C3091241C4217530721F5409195
:1040A000291C50912A1C2091251C3091261C421756
:1040B0005307C9F48FBFC150F9F61092B402FF91B3
:1040C000EF91CF91BF91AF919F918F917F916F9120
:1040D0005F914F913F912F910F900BBE0F900FBEAC
:1040E0000F901F9018954091291C50912A1C2091E7
:1040F000271C3091281C2150310942175307D1F257
:104100008FBF81E39CE10E94CF012FB7F894E0912B
:10411000291CF0912A1C80834091291C50912A1C53
:104120008091251C9091261C4817590751F48091C5
:10413000231C9091241C90932A1C8093291C2FBF30
:10414000BACF8091291C90912A1C0196F4CF80EC63
:1041500090E00E94760286E090E00E9476028091D4
:10416000301C90E00E94760280EC90E00C94760285
:1041700088E198E00FB6F894A895809360000FBE90
:10418000909360000E94EA050E940B06FBCF1F93EC
:10419000CF93DF93EC01162F0E94ED2B181739F007
:1041A000612FCE01DF91CF911F910C94F52BDF9100
:1041B000CF911F910895E1E3FCE11382128288EE12
:1041C00093E0A0E0B0E084839583A683B78386E480
:1041D00092E09183808385EC90E09587848784ECDE
:1041E00090E09787868780EC90E0918B808B81ECC4
:1041F00090E0938B828B82EC90E0958B848B86ECA5
:1042000090E0978B868B118E128E138E148E81E028
:104210008093CE1CEFECFCE11382128228E532E0A1
:104220003183208390E5948785878AE090E09787A3
:10423000868789E090E0918B808B82E090E0938B81
:10424000828B148A158A168A178A118E108E138E05
:10425000128E158E148E148215821682178208957E
:10426000CF93DF93CDB7DEB7C859D1090FB6F89415
:10427000DEBF0FBECDBF789484B5826084BD84B5A7
:10428000816084BD85B5826085BD85B5816085BD51
:1042900080916E00816080936E0010928100809109
:1042A0008100826080938100809181008160809391
:1042B0008100809180008160809380008091B100B6
:1042C00084608093B1008091B00081608093B000E1
:1042D0008091910082608093910080919100816033
:1042E00080939100809190008160809390008091F4
:1042F000A10082608093A1008091A10081608093E1
:10430000A1008091A00081608093A0008091210194
:10431000826080932101809121018160809321013D
:104320008091200181608093200180917A008460D7
:1043300080937A0080917A00826080937A008091E5
:104340007A00816080937A0080917A0080688093FF
:104350007A001092C10080917B00877F80937B0060
:1043600080E480937C0080917A00806480937A005E
:1043700080917A0086FDFCCF809178006091790071
:10438000762F682F072E000C880B990B611571058D
:104390008105910511F00E94C02AE4EFF5E081E06B
:1043A00094E0DF019C011D9221503040E1F7F09331
:1043B000241CE093231CF0932A1CE093291CF09307
:1043C000281CE093271C84EF99E09093261C80938F
:1043D000251CE091411CF091421C12E01083E091F9
:1043E0003D1CF0913E1C1082E0913F1CF091401C5E
:1043F00080E180831092491CE091451CF091461C9D
:1044000086E08083E091431CF091441C80818061B0
:104410008083E091431CF091441C808188608083FC
:10442000E091431CF091441C808180688083E0917E
:10443000431CF091441C80818F7D808310929000FA
:1044400089E18093910080E89EE3909397008093A8
:10445000960080E28093710061E08CE00E94580336
:1044600061E08DE00E945803E0E0F4E084EF91E029
:10447000DF019C011D9221503040E1F7E4E0FCE0B7
:1044800084E0DF011D928A95E9F7E8E0FCE080E036
:1044900090E1DF019C011D9221503040E1F7EEE5F3
:1044A000F3E082EADF01282F1D922A95E9F7F093C5
:1044B0001A1CE093191CF093201CE0931F1CF0932E
:1044C0001E1CE0931D1C2EEF33E030931C1C209328
:1044D0001B1CECEBF2E0DF011D928A95E9F7F093EB
:1044E0000C1CE0930B1CF093121CE093111CF09336
:1044F000101CE0930F1C8CE593E090930E1C8093AE
:104500000D1C8AE090E09093DE1C8093DD1C89E016
:1045100090E09093E01C8093DF1C82E090E0909309
:10452000E21C8093E11C2091F11C20FF6EC11093CE
:10453000BB028091BB028150823008F07BC283EDC8
:104540009FE00E943B1C833709F077C188E39FE01E
:104550000E943B1C833009F06CC189E39FE00E94FC
:104560003B1C8093BA02982F9F7B943A29F0993A8A
:1045700019F08F3F09F061C18AE39FE00E943B1C64
:1045800081508E3F08F059C18BE090E00E94742D5D
:104590006C018C0178E3E72E7FE0F72EC7010E94C3
:1045A0003B1CF80181938F01FFEFEF1AFF0A23E410
:1045B000E2162FE0F20691F780E190E00E94742D60
:1045C0008C0181E093E2A5E4B7E689879A87AB87FF
:1045D000BC8789E89BEAADECBFEE8D879E87AF87ED
:1045E000B88B8EEF9CEDAAEBB8E9898B9A8BAB8BDD
:1045F000BC8B86E794E5A2E3B0E18D8B9E8BAF8BFD
:10460000B88F1D821E821F821886FE01E75AFF4F57
:1046100080E4DF011D928A95E9F7CE018F5A9F4F02
:1046200028E0FC0111922A95E9F72BE0F601DE0162
:10463000599601900D922A95E1F720E82CA3FE01EE
:10464000B5962CE2DF011D922A95E9F748E550E086
:1046500060E070E049835A836B837C8328E5FC012A
:10466000208340E450E0BE01675E7F4F8055910992
:104670000E94800639852A859B858C85D8013C93CC
:1046800011962C93119712969C93129713968C93D4
:1046900013973D852E859F85888914963C931497A2
:1046A00015962C93159716969C93169717968C93A0
:1046B000179739892A899B898C8918963C93189772
:1046C00019962C9319971A969C931A971B968C936C
:1046D0001B973D892E899F89888D1C963C931C973A
:1046E0001D962C931D971E969C931E971F968C9338
:1046F0004801BB24B394C7010E943B1CF401919173
:104700004F018913B12CFFEFEF1AFF0A23E5E216E0
:104710002FE0F20681F7C8010E94102EC6010E9408
:10472000102EBB2009F48BC081E080932B1C8FEDF1
:104730009FE00E943B1C833709F081C084ED9FE01D
:104740000E943B1C90E09093FB0B8093FA0B85ED4D
:104750009FE00E943B1C90E090931502809314020E
:1047600086ED9FE00E943B1C90E09093170280939F
:1047700016028BED9FE00E943B1C182F8CED9FE0F2
:104780000E943B1C90E0B0E0A0E07C01DD24CC2442
:10479000F12A8DED9FE00E943B1C182F8EED9FE0CB
:1047A0000E943B1CC82AD12AC092000CD092010C56
:1047B000E092020CF092030C87ED9FE00E943B1CFC
:1047C000182F88ED9FE00E943B1C90E0B0E0A0E035
:1047D0007C01DD24CC24F12A89ED9FE00E943B1C62
:1047E000182F8AED9FE00E943B1CC82AD12AC09254
:1047F000FC0BD092FD0BE092FE0BF092FF0B82E1DE
:10480000809318020E94851C1AC022FF04C083E016
:104810008093BB028ECE23FF02C081E0F9CF42E23B
:1048200050E066E672E081E39CE10E9493010E9401
:1048300036068F7E803E09F490CE10922B1C992470
:104840009A94412C512C32015394AA24A39440E110
:10485000B42E8091301C882309F406C22FB7F89437
:104860008091F5099091F609A091F709B091F809A6
:104870002FBF4091F9095091FA096091FB0970919D
:10488000FC09841B950BA60BB70B0397A105B1057B
:1048900010F00E944D1A80912F1C882309F414C136
:1048A00010912E1C111102C00E944D1A80912D1CD6
:1048B0008111D6C180912C1C8111D2C1112331F0FC
:1048C00062E370E080E090E00E9485040E944D1A4F
:1048D00080912D1C8111F8C010922E1C8091F10B3B
:1048E0008111EAC081E08093F10B4FB7F8942091D9
:1048F0001D1C30911E1C80911F1C9091201C4FBFCD
:104900002817390709F4D8C0E0911D1CF0911E1C2E
:1049100080911B1C90911C1CE817F90709F091C0AD
:104920008091191C90911A1C90931E1C80931D1C41
:1049300080819181E0910F1CF091101C20910D1C41
:1049400030910E1CE217F30709F082C020910B1C76
:1049500030910C1C3093101C20930F1C008111818E
:10496000980121503109243F314008F0BECFADEF0E
:10497000B9E08D5F9940FC01EA0FFB1FFF70E85F13
:10498000F34F20812D939D012D5F39402017310772
:1049900090F38091301C882309F486C08091F90B34
:1049A00081115EC00E94EA050E94712AA301920152
:1049B0000E94032C607F862E0F3F110510F0689433
:1049C00080F890E080E00E942B19682D8FEC9CE12C
:1049D0000E94221C9DEFC92E99E0D92EEE24E3946B
:1049E000F12CD6016D916D018FEC9CE10E94221C8F
:1049F000BFEFEB1AFB0AEFEFEE16F10471F40E9421
:104A0000461890E080E00E942B19682D8FEC9CE105
:104A10000E94221CEE24E394F12CC6018D5F994084
:104A200080179107F0F20E9446180E94E6050E9446
:104A30003D1C5BCF10922B1C4EE150E069E872E008
:104A4000F2CEE0911D1CF0911E1CCF0102966CCF9E
:104A5000E0910F1CF091101C9F012E5F3F4F7ACF09
:104A60000E94EA050F3F110519F010F00FEF10E05A
:104A70008091F70B811116C090E080E00E942B1905
:104A8000BDEFEB2EB9E0FB2ED7016D917D018FECD0
:104A90009CE10E94221CC7018D5F994080179107FD
:104AA00098F3C1CFC801EACF82E00E94500585E0AB
:104AB00090E00E944D0619CF10922F1C1092181CE6
:104AC0001092171C1092F10B4FB7F8942091271CED
:104AD0003091281C8091291C90912A1C4FBF2817C7
:104AE000390709F4A3C481E08093221CFF24F394C6
:104AF000AEEFEA2E4FB7F8942091271C3091281C76
:104B00008091291C90912A1C4FBF2817390709F45E
:104B10008BC4E091271CF091281C8091251C90915A
:104B2000261CE817F90709F00EC18091231C90910B
:104B3000241C9093281C8093271C10818091211C99
:104B4000882309F476C4103C09F01EC18091190233
:104B5000811172C41092211C80911D1C90911E1C09
:104B60004091191C50911A1C8417950761F42091EB
:104B70001F1C3091201C80911B1C90911C1C28171D
:104B8000390709F4B7CF20911F1C3091201C809168
:104B90001D1C90911E1C02972817390709F4AACFF3
:104BA0008091171C9091181C8115904108F0A2CF9C
:104BB0002091151C3091161C8091131C9091141C8F
:104BC000019710F48FEF9FE02817390709F4C8C048
:104BD0002817390708F0BEC0821B930B0196009777
:104BE00009F488CF60912F1C6F5F60932F1CE091B8
:104BF0001F1CF091201C3183208360911F1C709139
:104C0000201C20911B1C30911C1C6217730709F09B
:104C1000AAC05093201C40931F1CE091111CF091DE
:104C2000121C918380832091111C3091121C809161
:104C30000D1C90910E1C2817390709F09FC0809118
:104C40000B1C90910C1C9093121C8093111C809152
:104C5000131C9091141C9093161C8093151C4ACF22
:104C600081E080932E1C30CF8091F30B9091F40B58
:104C7000A091F50BB091F60B0196A11DB11D2091ED
:104C80002B1C222379F1893FEAE29E07A105B10599
:104C900048F48093F30B9093F40BA093F50BB0932F
:104CA000F60B12CF1092F30B1092F40B1092F50B3F
:104CB0001092F60B6091CE1C623078F481E0809304
:104CC000F20B8091F20B680F6093CE1C70E08CE0C9
:104CD0000E9489030E94E605F7CE683290F3909215
:104CE000F20BEFCF893FFAE29F07A105B10558F417
:104CF0008093F30B9093F40BA093F50BB093F60B0A
:104D00000E94CD17E1CE1092F30B1092F40B10928B
:104D1000F50B1092F60B6091CE1C623078F481E0B6
:104D20008093F20B8091F20B680F6093CE1C70E0C1
:104D30008DE00E9489030E940B06E2CF683290F357
:104D40009092F20BEFCFE091271CF091281CCF013D
:104D50000196EFCEB501621B730B860F971F3FCFF5
:104D600081E090E03FCF20911F1C3091201C2E5FEE
:104D70003F4F3093201C20931F1C4FCF8091111C5C
:104D80009091121C02965FCF2091091C30910A1C51
:104D9000243F81E0380708F0ADCE9091190221152B
:104DA000310529F49E3F19F410931902A3CE9111F5
:104DB00044C01B3D19F4F092081C9CCE8091081C45
:104DC000882349F01C3D21F01D3D19F41BED01C065
:104DD00010EC1092081C80912F1C803508F08ACEB0
:104DE0008091171C9091181C8115904108F082CE7B
:104DF0008091171C9091181C01969093181C809319
:104E0000171C8091131C9091141C9C012F5F3F4F25
:104E10003093141C2093131C885F934FFC01108364
:104E20008091131C9091141C8115904109F062CE61
:104E30001092141C1092131C5DCE913009F04AC0E0
:104E40001B3DD9F49093081C8091091C90910A1C79
:104E5000049709F04FCE6091040C7091050C80917D
:104E6000060C9091070C0E94A42C61157105810518
:104E70009105D9F40E9478053DCE8091081C8823C5
:104E800049F01C3D21F01D3D19F41BED01C010EC53
:104E90001092081CC901019690930A1C8093091C6A
:104EA0002C5F334FD9011C93CFCF6093000C7093CC
:104EB000010C8093020C9093030C20911802213175
:104EC000C9F62091301C2223A9F20E947C170E946F
:104ED0004C19D0CF923009F048C01B3DD9F4F09264
:104EE000081C8091091C90910A1C049709F002CEBD
:104EF0006091040C7091050C8091060C9091070C48
:104F00000E94A42C6115710581059105D9F40E94B8
:104F10009D05F0CD8091081C882349F01C3D21F0AF
:104F20001D3D19F41BED01C010EC1092081CC901C5
:104F3000019690930A1C8093091C2C5F334FF90152
:104F40001083CFCF6093FC0B7093FD0B8093FE0B0F
:104F50009093FF0B809118028131C9F68091301C2B
:104F60008823A9F20E948519D2CF9330A9F41F3F5C
:104F700019F40E941A05BECD123108F011E1812FFB
:104F800090E090931702809316028091180281316D
:104F900081F70E94581CEDCF9430F9F41F3F19F4AB
:104FA0000E943E05A7CD86E090E0163038F0812FB4
:104FB00090E08D30910514F08CE090E09093FB0B25
:104FC0008093FA0B20911802213151F72091301C67
:104FD000222331F30E94AD18E3CF9530F9F41F3F3F
:104FE00019F40E942C0586CD85E090E0153038F04C
:104FF000812F90E08930910514F088E090E0909343
:1050000015028093140220911802213151F720914A
:10501000301C222331F30E94EB18E3CF9930B9F40E
:105020001093F80B112381F0F092F70B80EC90E0D5
:105030000E94760289E090E00E947602612F81E36F
:105040009CE10E9429022BC01092F70BEFCF963003
:1050500081F41F3F19F40E94A7204CCD111103C009
:105060000E94CD17F8CF113009F044CD0E94851C65
:10507000F2CF9132C9F480EC90E00E94760281E296
:1050800090E00E94760280E00E94640580E00E9429
:10509000640580E00E94640580E00E94640580EC65
:1050A00090E00E94760226CD923239F480EC90E0B6
:1050B0000E94760282E290E0E4CF933219F40E94DB
:1050C000D20518CD973081F40E94B80480EC90E0AE
:1050D0000E94760287E090E00E947602809113029F
:1050E00090E00E947602DBCF903329F4812F90E08C
:1050F0000E940F06FFCC903491F48091301C10E098
:10510000882331F06CE28FEC9CE10E94E917182FA4
:1051100080EC90E00E94760280E490E08DCF9830A1
:1051200071F4133709F0E6CC80EC90E00E9476022F
:1051300088E090E00E94760286E490E0D2CF9E3034
:10514000C1F4113089F41093F90B80EC90E00E94C7
:1051500076028EE090E00E9476028091F90B88231F
:1051600031F181E090E0BDCF1111EFCF1092F90B3A
:10517000ECCF9F30F9F480912F1C803580F4809122
:10518000171C9091181C8115904148F480EC90E018
:105190000E9476028FE090E00E947602E2CF80ECDF
:1051A00090E00E9476028FE090E00E94760290E00C
:1051B00080E097CF9935A9F4183F09F09BCC82E3A2
:1051C00090E00E944D0608E31FE06FEFC8010E94C7
:1051D000C7200F5F1F4F011520E11207B1F70E9492
:1051E000B820953521F4183F09F084CCF8CF9135DB
:1051F000B1F480EC90E00E94760281E590E00E949C
:10520000760208E31FE0C8010E943B1C0E9464056F
:105210000F5F1F4F011530E11307A9F740CF9235FB
:10522000D9F51B3DE9F4F092081C8091091C90917E
:105230000A1C029709F05ECC0091050C1091040C39
:1052400083ED9FE00E943B1C833711F1183C00F571
:10525000812F90E0602F885C904F0E94C7204ACC3D
:105260008091081C882349F01C3D21F01D3D19F454
:105270001BED01C010EC1092081CC901019690931F
:105280000A1C8093091C2C5F334FD9011C93CDCF8E
:1052900083E00E9450052ECC903579F480EC90E0AC
:1052A0000E94760280E590E00E94760281E090E024
:1052B0000E94760287E190E014CF983459F480EC94
:1052C00090E00E94760288E490E00E94760280E9F5
:1052D00090E007CF993459F480EC90E00E94760278
:1052E00089E490E00E94760282E990E0FACE93355C
:1052F00009F093C080912B1C882309F489C0809108
:10530000301C882309F484C06091FA0B84ED9FE07F
:105310000E94C7206091140285ED9FE00E94C72083
:105320006091160286ED9FE00E94C7206091FC0B01
:105330007091FD0B8091FE0B9091FF0B692F7727E9
:105340008827992787ED9FE00E94C7206091FC0B7A
:105350007091FD0B8091FE0B9091FF0BBC01882793
:10536000992788ED9FE00E94C7206091FC0B709107
:10537000FD0B8091FE0B9091FF0B672F782F892FEB
:10538000992789ED9FE00E94C7206091FC0B8AED70
:105390009FE00E94C7206091000C7091010C8091E9
:1053A000020C9091030C692F7727882799278BEDA2
:1053B0009FE00E94C7206091000C7091010C8091C9
:1053C000020C9091030CBC01882799278CED9FE07B
:1053D0000E94C7206091000C7091010C8091020C1A
:1053E0009091030C672F782F892F99278DED9FE0DF
:1053F0000E94C7206091000C8EED9FE00E94C720A4
:1054000063E78FED9FE00E94C7208AE090E070CEB6
:105410008AE090E00E94EE056DCB943509F06ACBEE
:1054200060E08FED9FE019CF1092221C0E949B023A
:1054300010CA103C09F05ECBF092211CE0921902D8
:1054400010920A1C1092091C55CB8F929F92AF921A
:10545000BF92CF92DF92EF92FF92CF93DF93EC0156
:10546000688179818A819B8161157105810591052A
:1054700021F464E279ED8BE597E02DE133EF41E033
:1054800050E00E94032C49015A019B01AC01A7EA9C
:10549000B1E40E94222C6B017C01ACEEB4EFA501BB
:1054A00094010E94302CC60ED71EE81EF91EF7FE8E
:1054B00006C081E0C81AD108E10880E8F80AC8826D
:1054C000D982EA82FB82C701B6019F77DF91CF9133
:1054D000FF90EF90DF90CF90BF90AF909F908F9014
:1054E00008958F929F92AF92BF92CF92DF92EF92E8
:1054F000FF9260911A0270911B0280911C029091A0
:105500001D02611571058105910521F464E279EDB3
:105510008BE597E02DE133EF41E050E00E94032C52
:1055200049015A019B01AC01A7EAB1E40E94222C77
:105530006B017C01ACEEB4EFA50194010E94302C0C
:10554000C60ED71EE81EF91EF7FE06C081E0C81A77
:10555000D108E10880E8F80AC0921A02D0921B0232
:10556000E0921C02F0921D02C701B6019F77FF90E6
:10557000EF90DF90CF90BF90AF909F908F90089565
:1055800060931A0270931B0280931C0290931D0279
:1055900008950E940B2B08F481E00895E89409C057
:1055A00097FB3EF490958095709561957F4F8F4F56
:1055B0009F4F9923A9F0F92F96E9BB279395F6956C
:1055C000879577956795B795F111F8CFFAF4BB0FEA
:1055D00011F460FF1BC06F5F7F4F8F4F9F4F16C04E
:1055E000882311F096E911C0772321F09EE8872FD8
:1055F000762F05C0662371F096E8862F70E060E094
:105600002AF09A95660F771F881FDAF7880F96950C
:10561000879597F90895990F0008550FAA0BE0E8B0
:10562000FEEF16161706E807F907C0F01216130664
:10563000E407F50798F0621B730B840B950B39F4A4
:105640000A2661F0232B242B252B21F408950A260A
:1056500009F4A140A6958FEF811D811D08950E9438
:10566000422B0C94B32B0E94A52B38F00E94AC2B3C
:1056700020F0952311F00C949C2B0C94A22B112458
:105680000C94E72B0E94C42B70F3959FC1F3950FE8
:1056900050E0551F629FF001729FBB27F00DB11DB6
:1056A000639FAA27F00DB11DAA1F649F6627B00D46
:1056B000A11D661F829F2227B00DA11D621F739F2F
:1056C000B00DA11D621F839FA00D611D221F749F3D
:1056D0003327A00D611D231F849F600D211D822F84
:1056E000762F6A2F11249F5750409AF0F1F08823AB
:1056F0004AF0EE0FFF1FBB1F661F771F881F9150D8
:105700005040A9F79E3F510580F00C949C2B0C94BF
:10571000E72B5F3FE4F3983ED4F386957795679542
:10572000B795F795E7959F5FC1F7FE2B880F911D01
:105730009695879597F9089597F99F6780E870E0A7
:1057400060E008959FEF80EC089500240A941616F7
:10575000170618060906089500240A94121613065F
:10576000140605060895092E0394000C11F48823ED
:1057700052F0BB0F40F4BF2B11F460FF04C06F5F09
:105780007F4F8F4F9F4F089557FD9058440F551FDF
:1057900059F05F3F71F04795880F97FB991F61F0B3
:1057A0009F3F79F087950895121613061406551F2A
:1057B000F2CF4695F1DF08C0161617061806991F96
:1057C000F1CF86957105610508940895E894BB278B
:1057D00066277727CB0197F90895F999FECF92BDF7
:1057E00081BDF89A992780B50895262FF999FECFA3
:1057F0001FBA92BD81BD20BD0FB6F894FA9AF99AEE
:105800000FBE01960895052E97FB1EF400940E948A
:105810001A2C57FD07D00E94352C07FC03D04EF4FC
:105820000C941A2C50954095309521953F4F4F4F31
:105830005F4F089590958095709561957F4F8F4F3C
:105840009F4F08950E94572CA59F900DB49F900DD7
:10585000A49F800D911D11240895B7FF0C94222C54
:105860000E94222C821B930B0895A1E21A2EAA1BE0
:10587000BB1BFD010DC0AA1FBB1FEE1FFF1FA21700
:10588000B307E407F50720F0A21BB30BE40BF50BFD
:10589000661F771F881F991F1A9469F76095709586
:1058A000809590959B01AC01BD01CF010895A29F09
:1058B000B001B39FC001A39F700D811D1124911DE4
:1058C000B29F700D811D1124911D08950E946D2CB1
:1058D0006894B1110C94E72B08950E94CC2B88F0AA
:1058E0009F5798F0B92F9927B751B0F0E1F0660FA4
:1058F000771F881F991F1AF0BA95C9F714C0B130E5
:1059000091F00E94E62BB1E008950C94E62B672FEE
:10591000782F8827B85F39F0B93FCCF38695779513
:105920006795B395D9F73EF49095809570956195FC
:105930007F4F8F4F9F4F0895EE0FFF1F881F8BBF24
:105940000790F691E02D1994692796276927782703
:10595000872778270895E894DF93CF93FC01DB0134
:105960000E94572C7F936F93E9019A01AC01BF937A
:10597000AF933F932F93DF010E94572C26F46C1BAB
:105980007D0B820B930B9E01EB01FC010E946B2DA2
:10599000AF91BF912F913F910E946B2DBE01CF011E
:1059A000F9012F913F91CF91DF910895689401C043
:1059B000E8948F929F92CF93DF930E94E42CDF9123
:1059C000CF919F908F90089588249924F401E40149
:1059D000B0E49F93AA279A158B049C04ED05FE055D
:1059E000CF05D007A10798F4AD2FDC2FCF2FFE2FC6
:1059F000E92D982C892E982F872F762F652F542FDD
:105A0000432F322F2227B85031F7BF9127C01B2ECA
:105A1000BF91BB27220F331F441F551F661F771FDF
:105A2000881F991F881C991CEE1FFF1FCC1FDD1FAC
:105A3000AA1FBB1F8A149B04EC05FD05CE05DF05DC
:105A4000A007B10748F08A189B08EC09FD09CE09A8
:105A5000DF09A00BB10B21601A94E1F62EF494013A
:105A6000AF01BE01CD01000C0895002E083090F06A
:105A7000982F872F762F652F542F432F322F2227D1
:105A80000850F4CF220F331F441F551F661F771F86
:105A9000881F991F0A95B2F7002D089597FD10945D
:105AA000002E083098F00850232F342F452F562F02
:105AB000672F782F892F912DF4CF1594979587957F
:105AC0007795679557954795379527950A95AAF73E
:105AD0001124002D08950E94572C460F571FC81FF0
:105AE000D91F08F4319608950F931F93CF93DF9336
:105AF0008230910510F482E090E0E091EF1CF0918B
:105B0000F01C30E020E0B0E0A0E0309799F42115DF
:105B1000310509F44AC0281B390B24303105D8F56A
:105B20008A819B816115710589F1FB0193838283D1
:105B3000FE0111C04081518102811381481759072C
:105B4000E0F04817590799F4109761F012960C93FA
:105B5000129713961C933296CF01DF91CF911F912C
:105B60000F9108950093EF1C1093F01CF4CF2115B2
:105B7000310551F04217530738F0A901DB019A01B2
:105B8000BD01DF01F801C1CFEF01F9CF9093F01C07
:105B90008093EF1CCDCFFE01E20FF31F8193919311
:105BA0002250310939832883D7CF2091ED1C3091C1
:105BB000EE1C232B41F420912002309121023093DE
:105BC000EE1C2093ED1C20911E0230911F02211526
:105BD000310541F42DB73EB7409122025091230286
:105BE000241B350BE091ED1CF091EE1CE217F3073E
:105BF000A0F42E1B3F0B2817390778F0AC014E5F3D
:105C00005F4F2417350748F04E0F5F1F5093EE1C6F
:105C10004093ED1C819391939FCFF0E0E0E09CCF07
:105C2000CF93DF930097E9F0FC0132971382128241
:105C3000A091EF1CB091F01CED0130E020E0109736
:105C4000A1F420813181820F931F2091ED1C3091AE
:105C5000EE1C2817390709F061C0F093EE1CE093A1
:105C6000ED1CDF91CF910895EA01CE17DF07E8F52B
:105C70004A815B819E0141155105B1F7E901FB8322
:105C8000EA8349915991C40FD51FEC17FD0761F4C0
:105C9000808191810296840F951FE9019983888301
:105CA000828193819B838A83F0E0E0E012968D915C
:105CB0009C9113970097B9F52D913C911197CD01C7
:105CC0000296820F931F2091ED1C3091EE1C281735
:105CD000390739F6309751F51092F01C1092EF1CED
:105CE000B093EE1CA093ED1CBCCFD383C283408144
:105CF0005181840F951FC817D90761F44E5F5F4F1C
:105D000088819981480F591F518340838A819B81E3
:105D1000938382832115310509F0B0CFF093F01CF5
:105D2000E093EF1C9ECFFD01DC01C0CF13821282F5
:065D3000D7CFF894FFCF6D
:105D3600FFDCFEB704B704B704B704B704B704B76B
:105D460004B704010500FF0011FE01000000000079
:105D5600F21C8000781E00A02800F03C0040510094
:105D6600127A00E4A20024F40048E80190D003204F
:105D7600A1070000000029029301C0017B02F10186
:105D8600CF01E30100000000221CE71B381CED1ABE
:105D9600D91B141BEE1A4572726F722C20696E6441
:105DA600657465726D696E61746520626F6F7420CB
:105DB600766563746F720D0A004572726F722C20DD
:105DC600696E636F727265637420626F6F7420769A
:085DD6006563746F720D0A0091
:00000001FF
